:020000040000FA
:06000000E8EF16F012000B
:0600080004EF08F01200F5
:060018000CEF08F01200DD
:06100000E8EF16F01200FB
:021006001200D6
:0610080065EF10F012007C
:06101800B0EF10F0120021
:02101E000100CF
:0C102000EC2D0000E80000000D000000B6
:04102C00D9CFE6FF33
:10103000E1CFD9FFE6520F015F6B626A160E616E57
:101040009F0E5B6F7B0E606E648C5C6B000EE66EB9
:10105000E66AE66A540EE66E0F0EE66EBEEC16F019
:101060000B6E050EE15E0B50649CDF6ADF500B6E69
:101070000C6A080E0B5C000E0C5810E2DF50040DD9
:10108000F3CFE9FFF4CFEAFF000EE926020EEA22D1
:10109000EE6AEE6AEE6AEE6ADF2AE8D70F01160EF4
:1010A000536F62A602D06296FCD70101B06BB56B9C
:1010B000B66BB76B6498080EA86F020EA96F9E6B93
:1010C0009D6BE552E552E7CFD9FF1200D9CFE6FF7D
:1010D000E1CFD9FFE65201019D0507E164BA05D0D1
:1010E000626A60806088020E9D6F6250040B05E0AA
:1010F0006050040B02E06294B7D864A202D0A194BD
:1011000082D06250010B12E06050010B0FE08EDFC5
:101110000101040E9D6F0201200E026F020E036F8B
:10112000080E016F006B8C0E001362906250100B62
:1011300005E06050100B02E085D862986250400BC9
:1011400013E06050400B10E0010EE66EE66A000E00
:10115000E66EE66A730EE66EE66ABAEC14F00B6EA3
:10116000060EE15E0B50629C6250200B04E0605062
:10117000200B01E04DD86250020B13E06050020BCF
:1011800010E0010EE66EE66A000EE66EE66AE668BC
:10119000E668BAEC14F00B6E060EE15E0B500F0120
:1011A0005F6B040E0101E76E9D19E8AE02D0E734D3
:1011B00002D0E7509D5D02E2A19425D060A622D026
:1011C000DF6A040EDF5C1EE262A61BD063CFBDF1B6
:1011D0006296780E0101BD1502E15BD810D0000EB9
:1011E000E66EE66ABD0EE66E010EE66E720EE66E05
:1011F000E66ABAEC14F00B6E060EE15E0B50DF2AC5
:10120000E0D700D0A194E552E552E7CFD9FF120014
:101210000F0153A115D0A0C1E9FFA1C1EAFFEF5012
:1012200080080DE1A8C1E9FFA9C1EAFFEF508408D9
:1012300006E1A0C1E9FFA1C1EAFF8C0EEF6E539158
:10124000629A1200608462986482000EE66EE66A1A
:10125000E66EE66A750EE66EE66ABAEC14F00B6EA0
:10126000060EE15E0B501200000EE66EE66AE66EB8
:10127000E66A740EE66EE66ABAEC14F00B6E060EC1
:10128000E15E0B506492609462A402D06294FCD739
:101290001200D9CFE6FFE1CFD9FFE652FD0E0101E2
:1012A000BD155AE17E0EBD15E8407F0B040DF3CF4E
:1012B000A0F1F4CFA1F1000EA027020EA123A0C13E
:1012C000A2F1A1C1A3F1A275A0C1E9FFA1C1EAFFEA
:1012D000EF503C0BE842E8420D083CE1A0C1E9FFB9
:1012E000A1C1EAFF020EE926000EEA22EECF0BF0C2
:1012F000EFCF0CF0280E0B1802E1020E0C1828E1BB
:10130000A0C1E9FFA1C1EAFF020EE926000EEA2210
:10131000200EEE6E020EED6EDF6ADF500B6E0C6A71
:10132000080E0B5C000E0C5813E2DF50EA6A280F1F
:10133000E96E020EEA22EF50E66EDF50EA6A200FF5
:10134000E96E020EEA22E552E750EF6EDF2AE5D79A
:101350000DD801D02ED805D0FD0EBD15040801E131
:101360004ED8E552E552E7CFD9FF1200A8C1E9FFF8
:10137000A9C1EAFFEF50800B05E0A8C1E9FFA9C1B0
:10138000EAFFEF6A0101AC6BAD6BB16BB26BB06B96
:10139000B9D8000EE66EE66AE66EE66A030EE66E01
:1013A000E66ABAEC14F00B6E060EE15E0B502EEFFF
:1013B0000CF0020E0101AD5D02E1B0DB1FD06FD871
:1013C0000101BE511AE1A2C1E9FFA3C1EAFFEE5239
:1013D000080EEF6EA2C1E9FFA3C1EAFF020EE926E3
:1013E000000EEA22200EEE6E020EED6EA2C1E9FFA3
:1013F000A3C1EAFF8C0EEF6E01D0BE6B1200D9CFF5
:10140000E6FFE1CFD9FFE652A8C1E9FFA9C1EAFF93
:10141000EF50400B01E0010EDF6E0101A875080ED0
:101420009D5D0DE122C25CFF0F015C51000804E2EA
:101430000101100E9D6F03D00101040E9D6FAD05DB
:1014400028E1A8C1E9FFA9C1EAFF020EE926000EC2
:10145000EA22280EEE6E020EED6ED5DA020E0101C2
:10146000AC5D07E1A8C1E9FFA9C1EAFF840EEF6EF8
:101470000FD0DF5007E1A8C1E9FFA9C1EAFFC80EFC
:10148000EF6E06D0A8C1E9FFA9C1EAFF880EEF6E92
:1014900001D005D8E552E552E7CFD9FF1200D9CFE8
:1014A000E6FFE1CFD9FF020EE1260101AD6BA8C135
:1014B000E9FFA9C1EAFFEF6A040EA8190B6EA9C1E2
:1014C0000CF00BC0DEFF0CC0DDFFDECFE9FFDDCF8F
:1014D000EAFFEF6AB5AF0CD0B851B91107E005D0FB
:1014E000B9C1FAFF0101B851F96EFADF0101B59FE8
:1014F000020EE15C02E2E16AE552E16EE552E7CFFD
:10150000D9FF120002012051600BE842E842E84294
:10151000E842E842000901E058D021510C0A54E0A9
:101520000B0A43E00C0A35E0010A26E00B0A22E030
:10153000020A20E0030A1CE0080A10E0010A0CE09D
:101540000F0A08E0030A01E03FD00101B08F080E46
:101550009D6F3BD0C8D839D07FDB37D001019E0EBC
:10156000AE6F010EAF6FB081010EB16FB08F2DD095
:1015700014D92BD02BD829D024510101AE6FAF6BD9
:101580009F0EAE27010EAF23B081010EB16FB08F59
:101590001CD00101B08F02012451EA6A9F0FE96E4D
:1015A000010EEA2222C2EFFF10D0000EE66EE66ABC
:1015B000E66EE66A020EE66EE66ABAEC14F00B6EB0
:1015C000060EE15E0B5001D000D01200D9CFE6FF2D
:1015D000E1CFD9FF040EE1260201220510E12051DE
:1015E0001F0B00090CE10101B08F030E0201215D08
:1015F00004E10101010EBC6F02D00101BC6B0201CC
:10160000225167E120511F0B020863E124510F0BA7
:1016100000095FE00101B08F020124BF10D0245106
:101620000F0BE96EEA6AD890E936EA36A40EE9268D
:10163000010EEA22EECFDEFFEDCFDDFF0FD0245109
:101640000F0BE96EEA6AD890E936EA36A80EE92669
:10165000010EEA22EECFDEFFEDCFDDFF030E215DAE
:1016600007E1DECFE9FFDDCFEAFF840EEF6E31D078
:1016700024510F0B0C6A530F0B6E0F0E0C22020E2F
:101680000BC0DBFF030E0CC0DBFF020EDBCFE9FF5C
:10169000030EDBCFEAFFEE90ED5224AF0DD0DECF8C
:1016A000E9FFDDCFEAFFEF6ADF74DECFE9FFDDCFD0
:1016B000EAFF400EEF6E0DD0DECFE9FFDDCFEAFF8F
:1016C000880EEF6EDF74DECFE9FFDDCFEAFFC80ED4
:1016D000EF6E040EE15C02E2E16AE552E16EE55272
:1016E000E7CFD9FF1200800E0201205D55E1010114
:1016F000C00EB06F02012351030A2EE0010A0EE072
:10170000030A03E00101B06B47D00101DC0EAE6FAC
:101710002B0EAF6F120EB16FB26B3ED02251F66E30
:10172000F76AD890F636F736800EF6262C0EF7229A
:101730000900F5CFAEF10A00F5CFAFF1020E0101BD
:10174000F76AAE25F66EAF51F7220900F5CFB1F179
:101750000A00F5CFB2F120D0030E225D1AE2225129
:10176000F66EF76AD890F636F736820EF6262C0E0D
:10177000F7220900F5CFAEF10A00F5CFAFF1AEC107
:10178000F6FFAFC1F7FF0800F5500101B16FB26B72
:1017900002D00101B06B00D01200D9CFE6FFE1CF3B
:1017A000D9FF020EE1260201286B296B20511F0B85
:1017B000020A12E0030A0DE0010A01E03BD0010138
:1017C000B08F020128810101BC0502E102012883DA
:1017D00031D00101B08F2ED00101B08F020124BFA2
:1017E00010D024510F0BE96EEA6AD890E936EA3638
:1017F000A40EE926010EEA22EECFDEFFEDCFDDFFDB
:101800000FD024510F0BE96EEA6AD890E936EA3618
:10181000A80EE926010EEA22EECFDEFFEDCFDDFFB6
:10182000DECFE9FFDDCFEAFFEF50040B02E0010E4F
:10183000286F00D00101B0AF07D0280EAE6F020EA6
:10184000AF6FB081020EB16F020EE15C02E2E16A9D
:10185000E552E16EE552E7CFD9FF1200649801012D
:10186000B0BF4AD0B5AF28D0020EAD6FA8C1E9FF16
:10187000A9C1EAFFEE52EF6AA8C1E9FFA9C1EAFFD8
:10188000C80EEF6EA2C1E9FFA3C1EAFFEE52080E37
:10189000EF6EA2C1E9FFA3C1EAFF020EE926000E26
:1018A000EA22280EEE6E020EED6EA2C1E9FFA3C180
:1018B000EAFFC80EEF6E1FD0A2C1E9FFA3C1EAFF85
:1018C000EE52080EEF6EA2C1E9FFA3C1EAFF020EBD
:1018D000E926000EEA22200EEE6E020EED6EA2C187
:1018E000E9FFA3C1EAFF8C0EEF6EA8C1E9FFA9C111
:1018F000EAFF840EEF6E86D0B5BF84D0020120AF20
:1019000059D00101B1510201265D0101B25102011C
:10191000275904E226C2B1F127C2B2F174D80101FD
:10192000010EAD6FA2C1E9FFA3C1EAFFEE52080E9E
:10193000EF6EA2C1E9FFA3C1EAFF020EE926000E85
:10194000EA22200EEE6E020EED6EA2C1E9FFA3C1E7
:10195000EAFF800EEF6EBE6BA0C1E9FFA1C1EAFFF6
:10196000EE52080EEF6EA0C1E9FFA1C1EAFF020E20
:10197000E926000EEA22200EEE6E020EED6EA0C1E8
:10198000E9FFA1C1EAFF840EEF6E010EBE6FA8C190
:10199000E9FFA9C1EAFF020EE926000EEA22280E9D
:1019A000EE6E020EED6EA8C1E9FFA9C1EAFFC80EF6
:1019B000EF6E28D00101020EAD6FA8C1E9FFA9C1E9
:1019C000EAFFEE52EF6AA8C1E9FFA9C1EAFFC80E1B
:1019D000EF6EA2C1E9FFA3C1EAFFEE52080EEF6E5F
:1019E000A2C1E9FFA3C1EAFF020EE926000EEA2226
:1019F000280EEE6E020EED6EA2C1E9FFA3C1EAFF52
:101A0000C80EEF6E1200D9CFE6FFE1CFD9FF020E6C
:101A1000E1260101080EB15D000EB2590EE2B1C11E
:101A2000DEFFB2C1DDFFAC5103E1010EAC6F04D0AB
:101A3000AC0502E1020EAC6F03D0080EDE6EDD6A6B
:101A4000A8C1E9FFA9C1EAFFEF92A8C1E9FFA9C1B6
:101A5000EAFFEF90A8C1E9FFA9C1EAFF010EDB5040
:101A6000EF12A8C1E9FFA9C1EAFFEE52DFCFEFFFF5
:101A7000000EDB50B15F010EDB50B25B280EBA6F77
:101A8000020EBB6FB0B121D0D9CFE9FFDACFEAFFA8
:101A9000EE50ED1019E0AEC1F6FFAFC1F7FFAE2B6F
:101AA000000EAF230800F550E66EBAC1E9FFBBC1D6
:101AB000EAFFBA2B000EBB23E552E750EF6EDF06BC
:101AC000010E01E2DB06E0D71FD0D9CFE9FFDACF64
:101AD000EAFFEE50ED1018E0AEC1E9FFAFC1EAFF3A
:101AE000AE2B000EAF23EF50E66EBAC1E9FFBBC1CB
:101AF000EAFFBA2B000EBB23E552E750EF6EDF067C
:101B0000010E01E2DB06E1D7020EE15C02E2E16ACE
:101B1000E552E16EE552E7CFD9FF1200D9CFE6FFDB
:101B2000E1CFD9FF020EE126A0C1E9FFA1C1EAFF82
:101B3000EE52EFCFDFFFDFCF0BF00B500101B65DB0
:101B4000000EB75903E2B6C1DFFF09D0DF500B6EBC
:101B50000C6A0B50B65DB66F0C50B759B76F010EDB
:101B6000DB6ADF50F36E010EDBCFF4FFF350F45C61
:101B700016E2010EDB50EA6A280FE96E020EEA2235
:101B8000EF50E66EB3C1E9FFB4C1EAFFB32B000E1C
:101B9000B423E552E750EF6E010EDB2AE2D7000EC8
:101BA000D880B655000EB75528E2A2C1E9FFA3C1FF
:101BB000EAFFEE52080EEF6EA2C1E9FFA3C1EAFFF1
:101BC000020EE926000EEA22280EEE6E020EED6EDF
:101BD000A0C1E9FFA1C1EAFFEF50400B07E1A2C19C
:101BE000E9FFA3C1EAFFC80EEF6E06D0A2C1E9FF6C
:101BF000A3C1EAFF880EEF6E25D0A2C1E9FFA3C101
:101C0000EAFFEE52080EEF6EA2C1E9FFA3C1EAFFA0
:101C1000020EE926000EEA22200EEE6E020EED6E96
:101C2000A2C1E9FFA3C1EAFF840EEF6EB851B9115A
:101C300007E005D0B9C1FAFF0101B851F96EFADF2A
:101C40000101B59F020EE15C02E2E16AE552E16E3C
:101C5000E552E7CFD9FF12000101B08F000EE66E0A
:101C6000E66AE66A540EE66E0F0EE66EBEEC16F0FD
:101C70000B6E050EE15E0B50010EE66EE66AE66A3B
:101C80009F0EE66E010EE66EBEEC16F00B6E050EB4
:101C9000E15E0B5022C29EF101019E5103E1100E44
:101CA0009D6F12D0200E9D6F010EE66EE66A9E0EAD
:101CB000E66E010EE66E010EE66EE66ABAEC14F010
:101CC0000B6E060EE15E0B501200D9CFE6FFE1CF9E
:101CD000D9FF020EE126000EDE6E020EDD6EFD0E55
:101CE000DB50E8240D6EFE0EDB50040DF3500D2486
:101CF000040DF3500B6E0C6A020E0F0B05E0D8902A
:101D00000C320B32E806FBE1D8900B360C36D8903B
:101D10000B360C36D9CFE9FFDACFEAFF0B50EE26AF
:101D20000C50ED22DECFE9FFDDCFEAFFEF9EFD0E86
:101D3000DB500FE1FE0EEA6ADB34FE0BEA36E96E99
:101D4000A40EE926010EEA22DECFEEFFDDCFEDFF85
:101D50000ED0FE0EEA6ADB34FE0BEA36E96EA80E00
:101D6000E926010EEA22DECFEEFFDDCFEDFFDECF6A
:101D7000E9FFDDCFEAFFEF9CDECFE9FFDDCFEAFF31
:101D8000040EE926000EEA22EF8C020EE15C02E26C
:101D9000E16AE552E16EE552E7CFD9FF1200D9CFF3
:101DA000E6FFE1CFD9FF020EE126FE0EDB500C6A02
:101DB000530F0B6E0F0E0C220BC0DEFF0CC0DDFFAD
:101DC000DECFE9FFDDCFEAFFFD0EDBCFEFFFDBA4C7
:101DD00007D0E66AFE0EDBCFE6FF77DFE552E5527D
:101DE000FD0EDBA208D0010EE66EFE0EDBCFE6FF95
:101DF0006CDFE552E552020EE15C02E2E16AE55277
:101E0000E16EE552E7CFD9FF1200D9CFE6FFE1CF6F
:101E1000D9FF020EE126FE0EDB5020E1A2C1E9FF50
:101E2000A3C1EAFFEE52080EEF6EA2C1E9FFA3C103
:101E3000EAFF020EE926000EEA22200EEE6E020EE6
:101E4000ED6EA2C1E9FFA3C1EAFF8C0EEF6EA8C13F
:101E5000E9FFA9C1EAFF840EEF6E3DD0FD0EDB5015
:101E6000E8240D6EFE0EDB50040DF3500D24040D1E
:101E7000F3CF0BF0F4CF0CF0000E0B26020E0C2269
:101E80000BC0DEFF0CC0DDFF840E0B6EDECFE9FF62
:101E9000DDCFEAFF0B50EF12FD0EDB50E8240D6E94
:101EA000FE0EDB50040DF3500D24010F040DF3CF93
:101EB0000BF0F4CF0CF0000E0B26020E0C220BC020
:101EC000DEFF0CC0DDFF840E0B6EDECFE9FFDDCF41
:101ED000EAFF0B50EF12020EE15C02E2E16AE5520A
:101EE000E16EE552E7CFD9FF1200D9CFE6FFE1CF8F
:101EF000D9FF020EE126FD0EDB500FE0FE0EEA6A6E
:101F0000DB34FE0BEA36E96EA80EE926010EEA2262
:101F1000EECFDEFFEDCFDDFF0ED0FE0EEA6ADB3442
:101F2000FE0BEA36E96EA40EE926010EEA22EECF98
:101F3000DEFFEDCFDDFFDECFE9FFDDCFEAFF020EF2
:101F4000E926000EEA22FB0EDBCFEEFFFC0EDBCF14
:101F5000EDFFDECFE9FFDDCFEAFFEE52FA0EDBCF79
:101F6000EFFF400E0B6EDECFE9FFDDCFEAFF0B5037
:101F7000EF16880E0B6EDECFE9FFDDCFEAFF0B50C8
:101F8000EF12FD0EDB500CE0FE0EEA6ADB34FE0BB6
:101F9000EA36E96EA80EE926010EEA22EF740BD0AC
:101FA000FE0EEA6ADB34FE0BEA36E96EA40EE92681
:101FB000010EEA22EF74DECF0BF0DDCF0CF00BC088
:101FC000F3FF0CC0F4FF020EE15C03E200D0E16A13
:101FD000E552E16EE552E7CFD9FF1200D9CFE6FF17
:101FE000E1CFD9FF64A84ED0FE0EEA6ADB34FE0BC7
:101FF000EA36E96EA80EE926010EEA22EE50EFCF8E
:10200000EAFFE96E400EEE16EE6AEE6AEE6AFE0E2A
:10201000EA6ADB34FE0BEA36E96EA80EE926010E09
:10202000EA22EE50EFCFEAFFE96EEE7CFE0EEA6A9E
:10203000DB34FE0BEA36E96EA80EE926010EEA2231
:10204000EF74400E0B6EFE0EEA6ADB34FE0BEA36CE
:10205000E96EA80EE926010EEA22EE50EFCFEAFF64
:10206000E96E0B50EF16FE0EEA6ADB34FE0BEA3621
:10207000E96EA80EE926010EEA22EE50EFCFEAFF44
:10208000E96EEF7CE552E7CFD9FF120005D0646A14
:10209000606A01019D6B00D0120001019D5114E1A5
:1020A000646A606A160E616E0F019F0E5B6F7B0E95
:1020B000606ED08EA284A084F28E64B602D0648654
:0A20C000FCD70101010E9D6F120014
:0620CA00DACFE4FFE2CFD3
:1020D000DAFFE9CFE4FFEACFE4FFF6CFE4FFF7CF82
:1020E000E4FFF5CFE4FFF3CFE4FFF4CFE4FFFACF52
:1020F000E4FF00EE00F00B0EE80403E3EECFE4FF94
:10210000FBD700EE0BF0030EE80403E3EECFE4FF91
:10211000FBD7E65266EC08F0E55200EE0DF0030E38
:10212000E80403E3E5CFEDFFFBD700EE0AF00B0E6A
:10213000E80403E3E5CFEDFFFBD7E5CFFAFFE5CFFA
:10214000F4FFE5CFF3FFE5CFF5FFE5CFF7FFE5CFF0
:10215000F6FFE5CFEAFFE5CFE9FFE5CFDAFF1100B3
:10216000D8CFE4FFE0CFE4FFE46EDACFE4FFE2CFC4
:10217000DAFFE9CFE4FFEACFE4FFF6CFE4FFF7CFE1
:10218000E4FFF5CFE4FFF3CFE4FFF4CFE4FFFACFB1
:10219000E4FF00EE00F00B0EE80403E3EECFE4FFF3
:1021A000FBD700EE0BF0030EE80403E3EECFE4FFF1
:1021B000FBD7E65294DAE55200EE0DF0030EE80488
:1021C00003E3E5CFEDFFFBD700EE0AF00B0EE804CA
:1021D00003E3E5CFEDFFFBD7E5CFFAFFE5CFF4FF53
:1021E000E5CFF3FFE5CFF5FFE5CFF7FFE5CFF6FF4E
:1021F000E5CFEAFFE5CFE9FFE5CFDAFFE550E5CF30
:10220000E0FFE5CFD8FF100006D84DEC10F0F28CBF
:1022100064D8FED71200D9CFE6FFE1CFD9FFE6524E
:1022200044D8DF6A100EDF5C0DE2EA6ADF34FE0B91
:10223000EA36E96E600EE926000EEA22EE6AED6AE1
:10224000DF2AF0D7DF6A5E0EDF5C15E2030EDF24C3
:10225000A96EA69EA69CA680DF5003E1A8CFEDF054
:1022600008D0DF04EA6A400FE96E010EEA22A8CF27
:10227000EFFFDF2AE8D75D0EE66EE66A400EE66EF7
:10228000010EE66E800EE66E000EE66E93EC16F022
:102290000B6E060EE15E0B50EDC0ECF016EC08F094
:1022A000E552E552E7CFD9FF120092680F0E936E08
:1022B000946A8A6A810ECD6E0A0EBD6E9F94320EAC
:1022C000C66EC76AB00EBA6E7F6A7E6A0001E86B9E
:1022D000E96BEA6BEB6B9D841200D9CFE6FFE1CF8F
:1022E000D9FF020EE126C0DA0001EE5101E0A5D0CF
:1022F000F0C0EEF00F0EEF25EA6A800FE96E000ED7
:10230000EA22EF5004E00001DE51400B1AE0000128
:10231000DE9DDEAF14D0DE9F5D0EE66EE66A400EF7
:10232000E66E010EE66E800EE66E000EE66E93EC33
:1023300016F00B6E060EE15E0B50EDC0ECF00001E6
:10234000EF6B0001DE91010EDB6A100EF36E010EE1
:10235000DBCFF4FFF350F45C6DE2010EDB500001C3
:10236000EF25EA6A800FE96E000EEA22EFCFDFFF69
:10237000DF5002E10001DE810001DEA113D0010E79
:10238000DBCFE6FF0F0EE552D880E754E96EEA6A2C
:10239000D890E936EA36600EE926000EEA22EE6AA7
:1023A000ED6A45D0200EDF5C03E3800EDF5C13E3B3
:1023B000010EDBCFE6FF0F0EE552D880E754E96E41
:1023C000EA6AD890E936EA36600EE926000EEA227B
:1023D000EE6AED6A2CD0200EDF5CF76A0A0FF66E0B
:1023E0002A0EF7220800F550F66EF76AD890F636F6
:1023F000F7366A0EF6262A0EF7220900F5CF0BF003
:102400000800F5CF0CF0010EDBCFE6FF0F0EE55212
:10241000D880E754E96EEA6AD890E936EA36600E69
:10242000E926000EEA220BC0EEFF0CC0EDFF010E04
:10243000DB2A8BD70001ECB1EF2B200E0101E76EF8
:102440009D19E8AE02D0E73402D0E7509D5D03E36A
:102450006450020B01E039D10001E851E91102E1B9
:10246000000E08D0E8C0E9FFE9C0EAFFEF50800B9A
:1024700001E0010E000901E028D102013651500AA5
:102480003CE0070A3AE0040A35E0010A01E00AD11B
:102490000001EA51EB1102E1000E08D0EAC0E9FFA9
:1024A000EBC0EAFFEF50800B01E0010E000921E1D3
:1024B0000201520E766F776B0001DEAF02D002018F
:1024C00077810001ECAF02D00201778F400EE66EFB
:1024D000760EE66E020EE66E010EE66EE66E75ECA8
:1024E0000FF00B6E050EE15E0B50F3CFEAF0F4CF68
:1024F000EBF0D8D037C2F0F0D5D037C2EDF0000104
:10250000400EE16F010EE26F0001EDA16DD0100EE3
:10251000E66EE66A200EE66EE1C0E6FFE2C0E6FF88
:10252000BEEC16F00B6E050EE15E0B50100E0001B6
:10253000E127000EE223010EDB6A3D0EF36E010E71
:10254000DBCFF4FFF350F45C22E2010EDB50020F0C
:10255000EA6A360FE96E020EEA22EF5001E117D067
:10256000010EDB50020FEA6A360FE96E020EEA2214
:10257000EF50E66EE1C0E9FFE2C0EAFFE12B000E9A
:10258000E223E552E750EF6E010EDB2AD6D70001B9
:10259000EDB315D0070EE66EE66A200EE66EE1C0DA
:1025A000E6FFE2C0E6FFBEEC16F00B6E050EE15E44
:1025B0000B50070E0001E127000EE22314D00F0E8E
:1025C000E66EE66A200EE66EE1C0E6FFE2C0E6FFD8
:1025D000BEEC16F00B6E050EE15E0B500F0E000107
:1025E000E127000EE22344D0100EE66EE66A200ECC
:1025F000E66EE1C0E6FFE2C0E6FFBEEC16F00B6E51
:10260000050EE15E0B500001EDB305D0080E000190
:10261000E127000EE223010EDB6A100EF36E010EBD
:10262000DBCFF4FFF350F45C23E2010EDB50020F2A
:10263000EA6A360FE96E020EEA22EF5001E118D085
:10264000010EDB50020FEA6A360FE96E020EEA2233
:10265000EF50E66E0001E1C0E9FFE2C0EAFFE12BC6
:10266000000EE223E552E750EF6E010EDB2AD5D7CC
:10267000E1C0E9FFE2C0EAFFEF6A0001DE8F00017E
:10268000EDA504D00001DE8D0001EE6B570E0201B6
:10269000365D07E1A69EA69CA6840001DD6B0001C5
:1026A000ED8F00D0400EE66E360EE66E020EE66E40
:1026B000E66A010EE66E75EC0FF00B6E050EE15E3C
:1026C0000B50F3CFE8F0F4CFE9F0020EE15C02E248
:1026D000E16AE552E16EE552E7CFD9FF12009D5065
:1026E000040B03E09E50040B01E1BDD0B00EBE26EA
:1026F000040EBF22070E0001F11557E10001F15150
:10270000E840E840E8401F0B0001E56F0001E5519B
:10271000030A3AE0010A27E0030A14E0010A01E093
:1027200044D08B868B820000000000000000000077
:1027300000000000000000000000000000008B927C
:102740008B9433D08B848B8200000000000000004B
:102750000000000000000000000000000000000079
:102760008B928B9A22D08B8A8B8200000000000013
:102770000000000000000000000000000000000059
:1027800000008B928B9811D08B888B820000000008
:102790000000000000000000000000000000000039
:1027A000000000008B928B9600D00001F1B11DD08B
:1027B0000F0E0B6E0001F151E8240C0B0001E52512
:1027C0000B5CE96EEA6AD890E936EA36600EE926D3
:1027D000000EEA22EECFE3F0EDCFE4F0C69EE4C0B7
:1027E0000BF00C6A0B50C96E03D0C69EE3C0C9FF44
:1027F0000001F1291F0B0001F16F0001F20708E150
:102800000001640EF26F0001EE5102E00001EE07DC
:102810000001EDAF27D0A6B225D03E0E0001DD5D50
:1028200004E3A6940001EC9F1DD0030E0001DD25FA
:10283000A96EAA6A0001DD5105E17F0E0001ED15C8
:10284000A86E09D00001DD05EA6A400FE96E010EAD
:10285000EA22EF50A86E550EA76EAA0EA76EA682AA
:102860000001DD2B9E94120000010A0EF35D000EA4
:10287000F45904E2500EF36FC30EF46FF307000E29
:10288000F45B64A205D0F351F41101E18B7040D0E8
:1028900001019D5102E18B903BD09D0502E18B80AF
:1028A00037D0020E9D5D0CE1020E0001F35F000EB9
:1028B000F45B0A0EF35D000EF45901E28B7028D030
:1028C000040E9D5D0CE1030E0001F35F000EF45B4E
:1028D0000A0EF35D000EF45901E28B7019D0100E50
:1028E0009D5D0CE1040E0001F35F000EF45B0A0E27
:1028F000F35D000EF45901E28B700AD0200E9D5D4D
:1029000007E100010A0EF35D000EF45901E28B703D
:10291000120012001200120012007CEF15F01200DB
:102920001E0EE66E010EE66ECFEC0EF0E552E5529D
:10293000400EE66E360EE66E020EE66EE66A010E9A
:10294000E66E75EC0FF00B6E050EE15E0B50F3CFEB
:10295000E8F0F4CFE9F0120064840001080EE66F9D
:10296000070EE76FE607000EE75BE651E711FAE1B5
:1029700064941200D9CFE6FFE1CFD9FFFD0EDBCF83
:1029800006F0FE0EDBCF07F0720E061801E10750CD
:1029900033E0E868061802E1E86807182BE0740ED7
:1029A000061801E1075024E0750E061801E10750F2
:1029B0001DE0730E061801E1075016E0030E06181D
:1029C00001E107500FE0020E061801E1075008E090
:1029D000010E061801E1075001E010D0A1DF0FD071
:1029E0009EDF0DD09ADF0BD096DF09D092DF07D0A3
:1029F00091DF05D091DF03D0000001D000D0010E9F
:0A2A000000D0E552E7CFD9FF120025
:062A0A00000000000000C6
:102A1000000000004443004200450203040506078D
:102A200008090A0B000000000000260C0D0E0F1014
:102A30001112131415161718191A1B1C1D1E1F200E
:102A4000212223242501010101012728292A2B2CD9
:102A50002D2E2F303132333435363738393A3B3C2E
:102A60003D3E3F4041010101010100007800E14885
:102A70000048610921498049A141E1418148E1497A
:102A80008149CF033F4AF3003F48F303C301FB02F0
:102A9000CC0300487C00C031F000CC14CC24FF00F3
:102AA000C703FF20C723BB030348FC00C090CCA092
:102AB00000B400543390F70A00046061E041600103
:102AC00060497081C101A045C041004020400078AC
:102AD0006000484308606041C0059045400120C047
:102AE00000436040408048A000B4005420810003AF
:082AF000004B00FC00903003D4
:082AF800020120511F0B01082F
:102B000001E06BD0245101E068D0060E215D28E180
:102B10002351230A21E0010A11E0030A01E020D039
:102B200001019E050AE10101000EAE6F2C0EAF6F90
:102B3000090EB16FB26BC00EB06F12D001019E05CD
:102B40000AE10101630EAE6F2C0EAF6F1D0EB16F67
:102B5000B26BC00EB06F04D00101800EB06F00D018
:102B600002012051600BE842E842E842E842E842B4
:102B7000010801E032D021510B0A29E0080A1CE0CB
:102B8000090A14E0080A07E00B0A04E0080A01E059
:102B900024D023D022D00101C30EAE6F010EAF6F3F
:102BA000010EB16FB26BC10EB06F17D00101800E74
:102BB000B06F23C2C3F111D00101C40EAE6F010E7C
:102BC000AF6F010EB16FB26B810EB06F06D0010115
:0C2BD000800EB06F22C2C4F100D01200D1
:042BDC0012010002E0
:102BE00000000008481A0333020001020001090234
:102BF0002900010100C032090400000203000000A6
:102C0000092111010001221D000705810340000177
:102C1000070501034000010403090430034B007958
:102C2000006F006800720069007400730075002076
:102C30000045006C00650063007400720069006369
:102C400000200049006E0064002E0018034B004273
:102C50000043002D005500530042006D0069006ED6
:102C60000069000600FF0901A101190129401500B2
:102C700026FF00750895408100190129409100C088
:082C8000EE2B172C1B2C4B2C32
:082C88001E0EF66E100EF76E31
:102C9000000EF86E00010900F550FA6F0900F550BA
:102CA000FB6F03E1FA6701D03DD00900F550F56FE5
:102CB0000900F550F66F0900F550F76F090009009B
:102CC000F550E96E0900F550EA6E090009000900A7
:102CD000F550F86F0900F550F96F09000900F6CFBB
:102CE000FCF0F7CFFDF0F8CFFEF0F5C0F6FFF6C030
:102CF000F7FFF7C0F8FF0001F85302E1F95307E0CE
:102D00000900F550EE6EF807F8E2F907F9D7FCC0B4
:102D1000F6FFFDC0F7FFFEC0F8FF0001FA07000E46
:062D2000FB5BBFD71200AF
:0A2D2600D9CFE6FFDACFE6FFFA0E80
:102D3000E3CFD9FFFB0EE3CFDAFFFC0EE3CFE9FFD1
:102D4000FD0EE3CFEAFFE9CFF3FFEACFF4FFF80E81
:102D5000E35003E1F90EE35008E0F80EE30602E267
:102D6000F90EE306DECFEEFFF2D7FF0EE3CFDAFF78
:102D7000E552FF0EE3CFD9FFE5521200FE0EE3CF7E
:102D8000E9FFFF0EE3CFEAFFE9CFF3FFEACFF4FF5D
:102D9000FB0EE35003E1FC0EE35009E0FB0EE306FB
:102DA00002E2FC0EE306FD0EE350EE6EF1D71200D8
:102DB000000EF36E00EE00F0030E01D81200EA6080
:102DC00002D0EE6AFCD7F350E9601200EE6AFCD73D
:102DD00011EE00F021EE00F0F86A0A9C44EC16F0C7
:0C2DE00003EC08F004EC11F0FBD712002B
:042DEC0000000000E3
:092DF00000000000320064000044
:020000040030CA
:0100000000FF
:0100010032CC
:0100020001FC
:010003001EDE
:0100050000FA
:0100060001F8
:0100080003F4
:01000900C036
:01000A0003F2
:01000B00E014
:01000C0003F0
:01000D0040B2
:0200000400F00A
:10000000000000012020202020202020202020206F
:10001000202020202A2A2031367365672044697306
:10002000706C617920436F6E74726F6C20627920FE
:100030004B42432D5553426D696E692056657231AE
:0B004000202A2A202020202020200061
:00000001FF
